:1000000083018B018A01850186018C019D018F018D
:100010009001910192019301940195019801990138
:100020009A01831610308500F03086008117640035
:10003000A730810083128501860105118510051006
:1000400027309E009F019F0B23289E0B23280F30F3
:1000500086053030860483160F300605860083122D
:10006000051505110B309E009F019F0B35289E0B37
:1000700035280515051101309E009F019F0B3E2874
:100080009E0B3E280F30860520308604051505118D
:100090002830822008308220013082200C308220DB
:1000A00006308220FE288316F030060486001830C1
:1000B0008500831285100514051505110608F03911
:1000C0009B0005150511060E0F391B049B1B5328B9
:1000D000051083160F30060586008312080096006F
:1000E00053200F3086051608F03986040510851454
:1000F000051505110F308605160EF0398604051515
:1001000005110800960053200F3086051608F039B7
:10011000860405108510051505110F308605160E8D
:10012000F03986040515051108009B010C089C0098
:10013000EB20031498020318A82803140130990235
:100140000318A828031401309A020318A8281B14C6
:100150009C031C08EB20031499020318B528031410
:1001600001309A020318B5281B149C031C08EB20CD
:1001700003149A020318BE280314BF281B0C003472
:100180009B010C089C00EB2003109807031CD3284C
:10019000031001309907031CD328031001309A077C
:1001A000031CD3281B149C031C08EB200310990785
:1001B000031CE028031001309A07031CE0281B14DD
:1001C0009C031C08EB2003149A07031CE928031462
:1001D000EA281B0C00348207003400340A3400344F
:1001E0000034643400340334E834003427341034E9
:1001F00001348634A0340F344234403411308C0042
:1002000009308D008E0106309D00952003180F29BE
:100210008E0A8D03031D052903308C021229C0208C
:1002200003308C0209308D0010301D079B009B03AA
:100230001B0884000E088E0180009D0301300C070E
:10024000031D052918088F0006309D0000308038F6
:1002500082200F301D078400000830386F200530E1
:1002600003151D02031D36292E306F209D0B2929F1
:100270000F301D078400000830386F204030803870
:10028000822020306F204D306F2048306F207A3030
:100290006F2000308038822097018101000000002B
:1002A0009D010B309E0001309F00D530A0008B01D6
:1002B0001030850083161F30850083120B1D6329C3
:1002C000970A0B1166290000000000009E0B5E29B2
:1002D0000B309E009F0B5E2901309F00A00B5E2912
:1002E000F4308E000B1D7729970A0B117A29000034
:1002F000000000008E0B72290000000000000000CA
:100300000000000000000000000003018600103023
:10031000850083161730850083120108990017089D
:100320009A009B019B0A851585110B110108031189
:100330001902031992299B0A9B099B0A1B0A980020
:02034000FE2895
:00000001FF
